:020000040000FA
:02000000852851
:08000800F000030EF1002030AE
:10001000A8002708A3002608A2002508A10024089C
:10002000A0000310A00DA10DA20DA30D031C8610AE
:100030000318861406191A28061D1C28A80B112857
:100040008B10710E8300F00E700E09009F1F0800C8
:100050000510061E2D288B1344288316E6309F00BA
:1000600083129F1F31288B133708A90000303C21D1
:100070003808A90001303C213908A90002303C2190
:100080003A08A90003303C2144281030AA00370860
:10009000AD003808AE003308B1003408B200642067
:1000A0002B08A4002C08A5001030AA003908AD00C8
:1000B0003A08AE003508B1003608B20064202B08BB
:1000C000A6002C08A70008002D08AF002E08B000DD
:1000D0000310B20CB10C3108AF02031C74283208B3
:1000E000B002031879287F28300803197F28B0034D
:1000F0006F282F08AD003008AE00031480280310CD
:10010000AB0DAC0DAA0B6428080003138316FD3059
:100110008600FE308500B7308100E7309F008312F3
:1001200005309F0000303621B70001303621B8007D
:1001300002303621B90003303621BA0004303621AE
:10014000B30005303621B40006303621B500073043
:100150003621B60045200B168B1705148519B328D8
:100160008619D828B6288619E928C728262085198F
:10017000C128861DB628861EBF280B21D828FA2044
:10018000D828051EC5282921C7281821C7282620B8
:10019000851DD228861DC728861ED0280B21E92858
:1001A000FA20E928051AD6282921B6281821B628C8
:1001B00026208519E3288619D828861AE1280B21DC
:1001C000B628FA20B628051EE7282921E928182193
:1001D000E9282620851DF4288619E928861AF228A0
:1001E0000B21C728FA20C728051AF8282921D82862
:1001F0001821D828B70A0319B80A34083802031995
:100200000629031C4528B701B801452833083702E1
:10021000031C4528032938083704031D1329340813
:10022000B8003308B700B7080319B803B703FD28AF
:10023000B90A0319BA0A36083A0203192429031C19
:100240004528B901BA01452835083902031C45285B
:1002500021293A083904031D31293608BA00350826
:10026000B900B9080319BA03B9031B2983169B0007
:100270001C141A088312080083169B008312290895
:1002800083169A001C1555309D00AA309D009C14C1
:0A0290009C1848291C118312080075
:02400E00623F0F
:104200004F000F00DB000300280017007800450076
:00000001FF
